S021000064656D6F70726F675F6F6C696D65785F73746D3332683130332E73726563A5
S3150800400000500020B9440008094500080945000881
S315080040100945000809450008094500080000000090
S31508004020000000000000000000000000094500082C
S315080040300945000800000000094500085145000828
S31508004040094500080945000809450008094500080A
S3150800405009450008094500080945000809450008FA
S3150800406009450008094500080945000809450008EA
S3150800407009450008094500080945000809450008DA
S3150800408009450008094500080945000809450008CA
S3150800409009450008094500080945000809450008BA
S315080040A009450008094500080945000809450008AA
S315080040B0094500080945000809450008094500089A
S315080040C0094500080945000809450008094500088A
S315080040D0094500080945000809450008094500087A
S315080040E009450008094500080945000800000000C0
S315080040F000000000000000000000000000000000B2
S3150800410000000000000000005FF808F1EE11AA5553
S3150800411010B5054C237833B9044B13B10448AFF3F3
S3150800412000800123237010BD00000020000000005D
S31508004130A845000808B5034B1BB103490348AFF36C
S31508004140008008BD0000000004000020A845000803
S3150800415000B583B00121102000F018F94FF4805300
S31508004160ADF8043003238DF8063010238DF8073098
S3150800417001A9034800F0B6F803B05DF804FB00BFD8
S315080041800010014010B500F0DDF90F4B1B68C31A8B
S31508004190B3F5FA7F0DD304460C4B1B7853B90122AD
S315080041A00A4B1A704FF48051094800F0ECF8064B98
S315080041B01C6010BD0022054B1A704FF4805104484C
S315080041C000F0DFF8F3E700BF200000201C00002005
S315080041D00010014082B00023019300932C4A136813
S315080041E043F4803313602A4B1B6803F400330093AF
S315080041F0019B01330193009B1BB9019BB3F5A06F8B
S31508004200F1D1234B1B6813F4003F06D0012300931A
S31508004210009B012B04D002B0704700230093F7E7F8
S315080042201C4B1A6842F010021A601A6822F0030240
S315080042301A601A6842F002021A60A3F580535A6897
S315080042405A605A685A605A6842F480625A605A68D4
S3150800425022F47C125A605A6842F4E8125A601A68C4
S3150800426042F080721A600A4B1B6813F0007FFAD07E
S31508004270074B5A6822F003025A605A6842F0020253
S315080042805A60034B5B6803F00C03082BF9D1C2E7AD
S31508004290001002400020024008B5FFF79BFF08BD4A
S315080042A008B50E4B1A6842F001021A6059680C4AA2
S315080042B00A405A601A6822F0847222F480321A6020
S315080042C01A6822F480221A605A6822F4FE025A609A
S315080042D04FF41F029A60FFF7DFFF08BD0010024087
S315080042E00000FFF8F0B4CB7803F00F02154613F080
S315080042F0100F01D08D7815430B78E3B106680023BB
S3150800430001E042610133072B14D801229A400C8838
S3150800431032EA0404F6D19C000F27A74026EA0706CE
S3150800432005FA04F42643CC78282CEAD0482CE9D19F
S315080043300261E7E706600B88FF2B20D94668002351
S3150800434002E0426115E00133072B17D803F1080490
S315080043500122A2400C8832EA0404F4D19C000F27FB
S31508004360A74026EA070605FA04F42643CC78282C43
S31508004370E7D0CC78482CE6D10261E4E74660F0BC89
S3150800438070470161704741617047000029B9054AC5
S31508004390936923EA000090617047024A93691843BB
S315080043A0906170470010024000B583B00023019366
S315080043B0009303F1804303F504331A6842F00102BF
S315080043C01A605968364A0A405A601A6822F0847296
S315080043D022F480321A601A6822F480221A605A6817
S315080043E022F4FE025A604FF41F029A601A6842F4D9
S315080043F080321A602B4B1B6803F400330093019B31
S3150800440001330193009B23B9019A40F2DC539A4287
S31508004410F0D1244B1B6813F4003F00D1FEE7224B72
S315080044201A6842F010021A601A6822F003021A602B
S315080044301A6842F002021A60A3F580535A685A6055
S315080044405A6842F400525A605A6842F480625A60C6
S315080044505A6822F47C125A605A6842F4E8125A6082
S315080044601A6842F080721A600E4B1B6813F0007FC0
S31508004470FAD00C4B5A6822F003025A605A6842F086
S3150800448002025A60074B5B6803F00C03082BF9D14C
S31508004490FFF75EFE00F040F803B05DF804FB00BFCE
S315080044A00000FFF8001002400020024008B5FFF7A0
S315080044B07BFFFFF767FEFCE7DFF834D0002103E057
S315080044C00C4B5B58435004310B480C4B42189A422C
S315080044D0F6D30B4A02E0002342F8043B094B9A4202
S315080044E0F9D3FFF7DDFE00F03BF8FFF7DFFF704773
S315080044F000500020C84500080000002000000020E9
S315080045000000002028000020FEE70000014B18608C
S31508004510704700BF2400002008B5074B074A5A60B9
S31508004520F021074A82F823100020986007221A60B3
S31508004530FFF7ECFF08BD00BF10E000E03F190100DF
S3150800454000ED00E0014B1868704700BF240000200A
S31508004550024A136801331360704700BF2400002025
S3150800456070B500250C4E0D4CA41BA410A54209D10C
S3150800457000F01AF800250A4E0A4CA41BA410A542FE
S3150800458005D170BD56F8253098470135EEE756F83F
S31508004590253098470135F2E7C0450008C0450008B0
S315080045A0C0450008C4450008F8B500BFF8BC08BCFB
S315080045B09E467047F8B500BFF8BC08BC9E467047D3
S309080045C0354100086B
S309080045C4114100088B
S705080044B9F5
